:020000000C28CA
:10000800FE000308FB000408FC000A08FD00472E58
:10001800512F00308A000408840A820700344334D0
:1000280041344D344F34E034A5344134A13448349C
:100038004F3443345434A5344B3441343A340034C7
:100048004234AE34A03445345034A53420344B34D3
:10005800413448344134A734203420342034003427
:100068005434453450344D344F344B344F34483481
:10007800543450344F34A734A73445345034003402
:1000880043344F345834503441344834A53454340C
:1000980062342034203448344534543400344834ED
:1000A80041344334543450344F34A6344B34A5349B
:1000B80020342034E03441340034203420342034D7
:1000C8004B34A734A5344D34413454342D34A5343D
:1000D80054340034A83450344F34AB34A534543439
:1000E800413448344F343A34003443344F3458346C
:1000F800503441344834453448344F343A34003469
:100108004334523443345F34443453343134383410
:100118002034003449344E34493454345F34443440
:10012800533431343834003420344F3454344B345D
:10013800A734B034AB344534483400344F345434E5
:100148004B34A734B034AB34A5345434623400345F
:10015800E03441345434AB34A5344B3420343D348A
:100168000034203442344B34A734B034AB344534F3
:100178004834003442344B34A734B034AB34A5345B
:100188005434623400344F34AC34A534A0344B3486
:10019800413420340034203445344334A734A53462
:1001A8002034543400344B34413448344134A73477
:1001B8002034003443345234433420344F344B34E5
:1001C800003445344534503452344F344D340034BF
:1001D8004B342E340034F9289829A029A529A029C0
:1001E800A529A629C6291E27CF29B401B501D908F2
:1001F800031D0329D80803193908031926290130D2
:100208004327C801C80A02303327B53043275908A5
:10021800031910297C30432758080319152972300F
:100228004327390803192429D33043273808C50040
:10023800C601BD254308122542081225410812258A
:10024800860108009A3043273108C6003008C500E7
:10025800BD254408303A031D3329203012253E08B5
:10026800031938292D3039292B3012254408303A02
:10027800031940294408122543081225420812256B
:100288002E3012254108122501301225433012253F
:100298002008CC002908CD002108CE000630CF0068
:1002A800D0012808B5222208CC002B08CD0023084D
:1002B800CE000630CF00D001D00A2A08B522240883
:1002C800CC002D08CD002508CE000630CF00023026
:1002D800D0002C08B5222608CC002F08CD0027080E
:1002E800CE000630CF000330D0002E08B522C8015A
:1002F800C80A02303327C5304327DB2112250130D5
:10030800D500360A89290310D50DFF3E031D87291C
:1003180055083F0503199229A330932986304327AE
:10032800BD0803190800942912304327DB21122540
:10033800BD08031908009C29EF21BD08031908000E
:10034800A129EF2932304327C801C80A02303327D0
:1003580041304327BC013B0BB8290B30C8000130A2
:10036800332703301225BC013A0BC2290B30C800D1
:100378000230332703301225BC01BC0ABD0803191B
:100388000800C2293C0BCA290130CB29003072234E
:100398000230BD0008004008840008300402031839
:1003A800080000308A00EF30040782000800360891
:1003B800D5003B08D5023A085507B600FB3036028F
:1003C800031CE8290330B600043036020318B601CE
:1003D8003608313E0800442AAC3043270B30C800A9
:1003E80001303327023012253608D0000310D00D13
:1003F8003B080319032A5008283E840080013A0864
:100408000319512A5008283E84008001800A512A85
:10041800AC3043270D30C800013033270230122595
:10042800023012253608D0000310D00D5008203EA7
:1004380084000008CA003B08CA023A084A07CB00F1
:100448005008203E84004B088000512A90304327F2
:100458000B30C80001303327023012250314360D43
:10046800D000FC29903043270D30C80001303327D5
:1004780002301225023012250314360DD0001A2A34
:100488004008023A0319F029013A03190C2A073ADD
:1004980003192A2A013A0319362A5008203E8400F3
:1004A8000008803AB73E500803185F2A203E8400AF
:1004B800C93080005008203E840000087F3A031DA0
:1004C8006A2A5008203E84007E308000C801C80A8D
:1004D80002303327DA3043273608313E1225BD3043
:1004E80043275008283E8400800803197D2A3E309F
:1004F8007E2A3C3012255008203E84000008CF0098
:10050800CF1F8B2A4F03FF3ACE002D30982A4F0871
:10051800CE005008203E84000008803A1C3E031C90
:10052800972A3130982A2B3012254E08C500C6016B
:10053800BD254208122541081225013012254330F5
:100548001225FF30CC001F30CD000130CC02003026
:10055800031CCD03CD024C0A03194D0A03190800E8
:10056800A92AD2000A30C500C6013108C8003008DF
:10057800C7001D264508D4003E080319C52AD4091A
:10058800D40A0130D100500ACB2A0310D10DFF3E06
:10059800031DC92A5108D3003F08D305D208031DFB
:1005A800EA2A4D080319EA2A5408803AD1004C086F
:1005B800803AD1020318E22AD301D30A4E08803ABE
:1005C800D1005408803AD102031CD3015208031900
:1005D800022BCD08031D022B4C08803AD100540889
:1005E800803AD1020318FA2AD301D30A5408803A70
:1005F800D1004E08803AD102031CD301D208031D52
:100608002C2BCD08031D2C2B4E08803AD1004C080A
:10061800803AD10254080318232B803AD1004C08A1
:10062800803AD10203182B2B4E08803AD100540887
:10063800803AD10203182B2BD301D30A2C2B803AF2
:10064800D1004C08803AD102031C202B182BD3016F
:1006580052080319562B4D080319562B4C08803A9B
:10066800D1004E08803AD1024C0803184D2B803A2D
:10067800D1005408803AD1020318552B5408803A07
:10068800D1004E08803AD1020318552BD301D30A62
:10069800562B803AD1005408803AD102031C4A2BC9
:1006A800422BD30153080130D1000319652B500A9E
:1006B8005F2B0310D10DFF3E031D5D2B5108BF04B6
:1006C8006F2B500A692B0310D10DFF3E031D672BBA
:1006D8005108FF3ABF053F0886000800CC008B137D
:1006E8001E27B901B7014C080319C22BCD01831687
:1006F8009C187B2B831203104D0D83169B008312CD
:100708004D08283E8400000883169A000524031823
:100718008B1783123708C5004D08283E840000084F
:10072800A62683169C18952B031483124D0D831649
:100738009B0083124D08203E8400000883169A000F
:10074800052403188B1783123708C5004D08203E6F
:1007580084000008A626CD0A08304D02031C7B2B16
:1007680083169C18B42B10309B008312370883160D
:100778009A00052403188B176730E32BCD0103106B
:100788004D0D83169B001C1483124D08283E11241E
:10079800283E84000008A62603144D0D83169B00EE
:1007A8001C1483124D08203E1124203E84000008AA
:1007B800A626CD0A08304D02031CC42B5C30432703
:1007C800103083169B001C141A088312B8003706D1
:1007D8000319F12BB901B90AF32BCC304327370899
:1007E800B800FF30CA00CB000130CA020030031C39
:1007F800CB03CB024A0A03194B0A031DF82B8B17AC
:10080800080003108B1B03148B131C1555309D0017
:10081800AA309D009C141C110800840083161A0835
:10082800800083123708C5004D080800FF30D60045
:10083800D7000130D6020030031CD703D702560A6E
:100848000319570A031D1D2C0827EF2522304327BB
:10085800C801C80A023033274F304327FF30D6007B
:10086800D7000130D602031CD703560A0319570ACA
:10087800031D352C0130D602031CD703560A031971
:10088800570A031D3E2C0130D6020030031CD70343
:10089800D702560A0319570A031D472C0030722342
:1008A800F72031083306031D5B2C30083206031984
:1008B800622C3108B3003008B200F7203D08031954
:1008C800852C752CBB01BB0A7F2CC00A083040025E
:1008D8000318C001BD0803197F2C6E2CBA01BA0A8F
:1008E8007F2C3D08013A0319662C033A0319692C39
:1008F800013A0319722CFF30B400B500F720BA0191
:10090800BB013508340403199B2C0130B402031CC5
:10091800B5030F30D600D7010130D6020030031CD2
:10092800D703D702560A0319570A031D902C34031C
:100938003504031D552CC001003072230430BD005E
:10094800552CF126CC30DA264430DA26F126CC3084
:10095800DA26BE30DA266926FA0083120313B701B5
:100968003708F1007A088926692683120313B00034
:10097800B1013708F100300889263008F8007A08F4
:10098800B0007808B100FA013708F1006926892615
:10099800FA0A06307A02031CC82C6926831203134C
:1009A8003706031DD92CD801DB2CD801D80A310809
:1009B800F9003008F80008300310F90CF80CFF3E75
:1009C800031DE02C10307802BE01031CF52CBE0A72
:1009D8000130F80030087802B00031090318013EF0
:1009E800B1000A30F000F1013108F3003008F200DC
:1009F800C1267108B1007008B000B00EB10E0F30FA
:100A0800B0053108F039B0040F30B1053108033AA8
:100A18005230031930060319D9010800C7000A30FB
:100A2800C6004708C50007300310C50CFF3E031D6C
:100A3800182D451C212D0515222D05114708C50027
:100A480006300310C50CFF3E031D252D451C2E2D19
:100A580085152F2D85114708C50005300310C50CD5
:100A6800FF3E031D322D451C3B2D05143C2D051062
:100A78004708C50004300310C50CFF3E031D3F2D79
:100A8800451C482D8514492D851085178513470861
:100A9800C5000310C50C0310C50C0310C50C451C7C
:100AA800572D0515582D05114708C5000310C50C0D
:100AB8000310C50C451C622D8515632D851147084B
:100AC800C5000310C50C451C6B2D05146C2D0510B5
:100AD800471C702D8514712D851085178513C60345
:100AE8004608FF3A03190800732D05135F301225D5
:100AF8000517003012250030122504301225023067
:100B080012251F301225023012250430122500301C
:100B1800122500301225043012250E30122515300A
:100B28001225043012250430122504301225043011
:100B38001225003012250030122500301225003011
:100B480012250030122506301225093012250630EC
:100B580012250030122500301225003012250030F1
:100B680012250030122500301225003012250030E1
:100B7800122D3030C100C200C300C4000330460249
:100B8800E83003194502031CD42DC40A1830C507E0
:100B98000318C60AFC30C607C22DC30A9C30E925D3
:100BA80000304602643003194502031CDF2DD12DA5
:100BB800C20AF630E925003046020A300319450218
:100BC8000318DC2D4508C1070800C5070318C60A25
:100BD800FF30C607080053308312CA000530CB0027
:100BE8000130CA02031CCB034A0A03194B0A031D2E
:100BF800F42D051305118511051485108517851326
:100C08007430CA000130CB000130CA020030031C26
:100C1800CB03CB024A0A03194B0A031D082E2B30BB
:100C28001225133012250C3012250430122579258F
:100C38001E2FC901CA01460845040319422ECB01DB
:100C4800CB0AC61B2B2E0310C50DC60D242E031070
:100C5800C90DCA0D46084802031D342E450847022F
:100C6800031C3E2E4508C7024608031CC803C802D9
:100C780049140310C60CC50CCB0B2B2E4A08C60012
:100C88004908C500080001300B1D00398B1E0039CA
:100C980000380319602E0B1183120313BD01861B44
:100CA800572EBD01BD0A061B5B2E0230BD00861AF9
:100CB8005F2E0330BD00A5247D088A007C088400CF
:100CC8007B088300FE0E7E0E0900F601F701770807
:100CD800083A0319872E8316031306128312061285
:100CE800831606168312061E842E0130F500770A35
:100CF8007F2E0310F50DFF3E031D7D2E7508F604AB
:100D0800F70A63276B2E76080800F300F4017108D0
:100D18007306F200721C972E031418307106F20045
:100D2800720CF1009A2E0310F10CF1130310F30C5E
:100D3800F40A083074027108031C8C2E8312031302
:100D4800B7000800C700C80145084706C600461C8A
:100D5800B42E031418304506C600460CC500B72E3D
:100D68000310C50CC5130310C70CC80A0830480285
:100D78004508031CA92EB7000800F401F501701CF2
:100D8800CB2E7208F4070318F50A7308F507031049
:100D9800F20DF30D0310F10CF00C71087004031D33
:100DA800C32E7508F1007408F0000800F100F20184
:100DB8007208083A031908008316031306128312EF
:100DC8000612711CE92E0616EA2E06120310F10C03
:100DD800F20A632783160616DC2E831603130612FF
:100DE800831206127730F000F0037008FF3A031DF3
:100DF800F82E8316031306164A30F000F003700825
:100E0800FF3A03190800022F8B0120308316850052
:100E1800E0308600073083129F0085018601831623
:100E28008113811281110115811401148B160B1184
:100E38008B170800B430C800C9010513013012250A
:100E48000130C8020030031CC903C902480A03194B
:100E5800490A031D242F8030122505170800C900F0
:100E68000513490B3A2F48087F3E12254908023AD4
:100E7800031D412F4808BF3E12250517080083129D
:100E8800C800480884000D201225C80A48088400B4
:100E98000D20003803190800452F831320308400E3
:100EA80045305B270130D800D90083011A2C640033
:100EB8008001840A04060319003404065C2F0A30F2
:0E0EC800F000F0037008FF3A03190800652FD0
:02400E00503F21
:1042000000000A0001001400010005000000FB008E
:104210000000140000000A000100140001000F005B
:10422000D3000000000000000000000000000000BB
:00000001FF
